:100000006F00106A000000004A0100004C0100006F
:1000100000000000000000000000000000000000E0
:1000200000000000000000000000000000000000D0
:100030009E0E0000000000009E0E00000000000068
:100040009E0E00009E0E00009E0E00009E0E000000
:10005000560600009E0E00009E0E00009E0E000040
:100060009E0E00009E0E00009E0E00009E0E0000E0
:100070009E0E00009E0E00009E0E00009E0E0000D0
:100080009E0E00009E0E00009E0E00009E0E0000C0
:100090009E0E00009E0E00009E0E0000000000005C
:1000A000511126C022C206C4828282441244A24058
:1000B000310182802A86014593F6150091C232955E
:1000C00085810606F5F9828000000000634E050276
:1000D00063C305042E86AA857D5515C285466378BF
:1000E000B6006356C00006068606E36CB6FE014500
:1000F00063E4C500918D558D85820582F5FA828075
:100100008682C93F2E8582823305A04063D70500D1
:10011000B305B040C1B7B305B0408682653F330533
:10012000A0408282868263C70500634905005D376F
:100130002E858282B305B040E35B05FE3305A04007
:10014000513F3305B0408282000001A0B707EFBEE7
:1001500037E700E0938707083CC701A07D15131718
:10016000050141839307F00363EBE700B707002025
:100170009387C701AA9788231375F50F82800145DD
:100180008280EFF2FFF1B7E700E03707100023A00D
:10019000E7180F100000EF00D06413051003EF0004
:1001A000D06637450008130505FCB7040020EF00B2
:1001B000D06901449384C401B38784008C239307DE
:1001C0001400A6979C2337450008130505FCA207D9
:1001D000DD8D2295EF00F06A090493070004E31D0A
:1001E000F4FCEF00B061E520B7E700E0370710004E
:1001F00023A0E7105DBDEFF2BFEAB7460008370461
:1002000000208147938606FC1304C40113060004F2
:100210003387D7001823B305F40085071377F70F4A
:1002200098A1E397C7FE7C301307F00F6312F70223
:10023000056781471307C74A930600043306F70092
:100240000C223306F40085070CA2E399D7FE153F74
:100250000347F403B707002085461377F70F93870A
:10026000870163E4E60098A389B523800700EDBF0A
:100270009307F5FF1397070141839307F00363E7A3
:10028000E704EFF2FFE1B7070020A1469387C7011B
:100290006317D5026395A502856601479386C64A12
:1002A00013060004B385E6008821B385E70005073F
:1002B00088A1E319C7FEF135EF00A06DFDB3BA9731
:1002C0009823E38DE5FE8CA36D3DCDBF8280EFF2D8
:1002D0003FDD23A40184239C0184A3820184238B1A
:1002E0000184B7070040DE331145C207C18323965E
:1002F000F184EF00704E55BBEFF29FDA1C210D47E1
:100300007111AA8493F7F70F6374B70A1831139425
:10031000870013740430598C9306400713F7470F76
:1003200005046312D702A18B99C7EF004077AC2078
:1003300022853D3F91A022851535BC20631EF50224
:10034000EF00E07515A893F7C70F130780076395B3
:10035000E7023C21228593F7F70F3EC00135B82014
:100360008247418B9D8B19EBB820B357F540858BA5
:100370000D83058BE386E7FC110105BB3EC0EF0052
:1003800000728247B8208544B394F400E204937766
:100390008700E184228591C7D133458D9375F50F90
:1003A00041BF6D3B93C4F4FFE98C93F5F40F49B75B
:1003B000E394E5FC13F7070F93060007E31ED7FA53
:1003C00013F777009546631AD7001C3137070020D2
:1003D00093F7F70F2300F700A5B793F647009DE2C8
:1003E000B706002003C506000A0575153A954205B3
:1003F000418159D1A18B95C72AC0EF00406A8C304A
:10040000024505BF9146630AD70099466309D700A4
:100410009D462145E312D7F6F1BF7545E1BF1D4565
:10042000D1BF2D3B9C3019BF83D7A1869DEFEFF242
:100430003FC704212A84054593F4F40F05336395DF
:10044000A4021C30094593F4F70F093B93F7E40F1E
:10045000631CF5000830B707002083C787010589B2
:100460006384A700EF00007289B18280EFF25FC35E
:10047000B307C5009C231307F00393F7F70F6397A7
:10048000E708130726006353B70805062A961822C3
:100490001C2285469354770013F4F707631ED4009B
:1004A000A38D0184238D018423860186B707002054
:1004B000A3809700C523B1A009C49307F4FF13F4E8
:1004C000F70FB706002083C62600639D960283C6F9
:1004D000B1858DEA0DC81305F002493109CD0546F5
:1004E0001305F0022386C1869539931625003695AB
:1004F00006052397A186B7070020A3809700238DC8
:10050000818465B66DF823860186F5B713F7070C6D
:1005100093060004631AD70693D657401397170023
:100520009187798B858BD98F1387E7FF1377F70F27
:10053000854593F41600E3F5E5F6014463F7F5000D
:100540009387D7038A0713F4F70FB707002083C7F1
:1005500027006397970283C7B1859DE31DC01305EC
:10056000F002ED3E49D905471305F0022386E186E6
:10057000F536131725003A9506052397A186A5BFE2
:100580003DF82386018685BF13F7070E9306000802
:10059000631AD70213D74740058B238EE18413D704
:1005A0003740058BA381E18613D72740058B238134
:1005B000E18613D71740058BA380E186858B2380C6
:1005C000F186CDBD13F7070F9306000B6315D70215
:1005D00013D73740058BA383E18613D72740058BBC
:1005E0002383E18613D71740058BA382E186858B91
:1005F0002382F186C1B59306000A6315D70213D78B
:100600003740058BA38FE18413D72740058B238FB9
:10061000E18413D71740058BA38EE184858B238457
:10062000F18649BD13F7C70F9306C00EE31BD7EC45
:1006300013073600E357B7EC130716002A97182361
:1006400009062A96139587000C2213750530598DDB
:10065000050539397DB57111114522C0EF00F0153E
:10066000630D050C1145EF003017B7070040DA3372
:100670009387C18482234207418333048740420425
:100680004180CD4663FB860A37150140914513052D
:1006900005809AA3EF00F0294DE109671307077160
:1006A000938781846377870023A00700239C0184BC
:1006B00069A0984385466305D70A25C38946E31593
:1006C000D7FE138661841822133414050607598C4B
:1006D0001374F40F9386418400A2982205071377C0
:1006E000F70F98A2A146631AD704938651849822E3
:1006F000954563E1E50298229375F70F138715007E
:100700001377F70F98A214221387018593F6F60F3B
:100710002E9714A3054798C30DA0930600051387D1
:10072000818563E086021E239306900F63E7F6003F
:100730001E238507C207C1831EA302441101730053
:10074000203016232546637AD600894694C3238237
:10075000018423830184A382018423100700F1BF55
:100760009306000563F98600094798C32382018434
:1007700023830184D9B7238BE18423A00700239C22
:10078000E18465BFEFF2DF91130141FC0545EF0005
:10079000B01DEF00006A8534A12485451305500281
:1007A000EF00302485653146138445480810938551
:1007B0004548EF00F03F371501400C101305058048
:1007C000EF00700F89450145EF00F0174146930592
:1007D000C4006810EF00D03D6810EF006077930709
:1007E00040117C86680085473EC823070100EF0062
:1007F000101885450545EF00B020B707002003A578
:100800004701B7450F0093850524EFF0BF8C7D1598
:10081000C167FD17E8824C08370500403ECC231B1A
:100820000100230E0100EF00901F854537050040B1
:10083000EF001034B7070040C23342044180B707CD
:100840000040DE331307703E818FC207C183637798
:10085000F7001304843E42044180E52183C761858B
:1008600093F7F70FE9DFB7E700E03707100023A0A1
:10087000E7180F10000083C55184814793F4F50FEA
:100880009386018513F6F70F63669604238B018424
:10089000A3820184B7E700E03707100023A0E71028
:1008A000814681471387F4FF63CEE7027C183E97A9
:1008B000834787FCE395D7F88947E3F297F81C82D2
:1008C0001307000793F6070F6397E602A685480013
:1008D0002534B5B73386D700082250003E9608A2CB
:1008E00085074DB770183E96034686FC850793F73B
:1008F000F70FB18E55BF93F7070C130700086395E8
:10090000E7004800153625BF7545EFF03F851375A4
:10091000050215C58D47E384F4F21C8245453EC0AF
:10092000EFF0DF838247E39CA7F09C8249453EC0FD
:10093000EFF0DF828247E394A7F0094611A81C82FA
:1009400005453EC0EFF09F8182470546E399A7EE3B
:10095000A6854800213EE5B5EFF28FF4B7070020E9
:1009600083C7870199EF0146894537150140EF009C
:10097000E07C0546914537150140EF00207C6FF083
:10098000CFF20546894537150140EF00207B01462F
:10099000D5B7EFF2EFF0B707002003A44701B7C7C0
:1009A000FA7B9387F74F814563F487000D809D455F
:1009B000B73401400546138504C0EF00501EA16501
:1009C000938505D02285EFF0EFF09305F5FFC20582
:1009D000C181138504C0EF00F01CBD3F6FF0EFEC48
:1009E000EFF20FEC130181FD854513055003EF0075
:1009F000407F0565854513050580EF00807E8547AE
:100A0000C1443EC86C0099473715014026CA7C8610
:100A100023170100EF00206A371501408947614420
:100A20006C00130505807C8622CAEF00C0686C004C
:100A300037150140648622CABD2D37340140930723
:100A4000B05D8A85130504C03EC202C023040100C4
:100A5000EF00E07CC167938707062C08130504C0EC
:100A60003ECC02CE02D002D2EF0050002C0813057B
:100A700004C0EF001009130504C08545EF00D01035
:100A80008545130504C0EF00B00E21371301810224
:100A90006FF0AFE1EFF2CFE0C1356FF00FE1EFF2B1
:100AA0002FE0B7070040D63305674111C206C18267
:100AB000B704004013077738DE30958FC207C18333
:100AC000E37CF7FE0546994537150140852D3734FF
:100AD00001408355C4C2130404C022858505C205A4
:100AE000C181EF00700C81452285EF00300CD630BB
:100AF000096737060040C206C1821307F7705E32ED
:100B0000958FC207C183E37CF7FE3734014013059C
:100B100004C08145EF005009130504C08145EF0072
:100B2000F008856531469385054A4800EF00500876
:100B3000371401404C0013050480B52BC1474C000D
:100B4000371501407C823EC0BD2313050480014659
:100B50008945ED230146C14537150140C5230947A5
:100B6000E1444C0013050480788226C6A9238247FD
:100B70004C00371501407C8226C6352BF13B4101E4
:100B80006FF0AFD2EFF2CFD101112AC01545EFF0CF
:100B9000EFDC931725003E95060542050567418168
:100BA00081471307F7F96398A7143734014081454B
:100BB000130504C0EF00407F8145130504C0EF001A
:100BC000E07E1307F01802C6B2476372F714B73716
:100BD0000140938407C0C2341945EFF02FD8420476
:100BE0004180A285EFF00FCD9305F00FEFF08FCE8F
:100BF000824742054181854613071400098C639C96
:100C0000D71093150701C1812685EF00E079931570
:100C10000401C1812685EF0060790D45EFF00FD406
:100C2000931725003E9506054205056741818147DA
:100C30001307F7F9639BA70E1145EFF02FD2058933
:100C40003DC937340140130504C08145EF00C0752C
:100C5000130504C08145EF006075856531469385B5
:100C6000054A4808EF00C074371401404C081305CA
:100C70000480912141474C0837150140F8823AC25F
:100C80001D2901468945130504804D290146C145AA
:100C90003715014065218947FC824C08E14713055F
:100CA00004803ECE09291247E1474C083715014020
:100CB000F8823ECE0921B707002003C7870182468C
:100CC000630CD700238CD700B70700209387C70198
:100CD000A38FD702EFF0EFCA2545EFF02FC8931787
:100CE0001500AA978E073E950A052395A186AD317A
:100CF00005616FF08FBB02C4A2466376D7008507FB
:100D0000C207C1834DB5A246850636C4F5B7B247C2
:100D100085073EC655BD93150401C18126853AC29B
:100D20006125124793150701EDB502C8C2466376E7
:100D3000D7008507C207C183F5BDC246850636C800
:100D4000F5B79387A1869A2319C37D179AA382804A
:100D5000EFF20FB5371402401C403707FFF841454A
:100D600093E717001CC05C40F98F5CC01C4037073C
:100D7000F7FE7D17F98F1CC01C403707FCFF7D175D
:100D8000F98F1CC05C4041777D17F98F5CC0B707B5
:100D90009F001CC435291C4C93E707021CCCB717D5
:100DA000014003A70740938607401377F7F023A07D
:100DB000E74003A707401367070823A0E7408947D8
:100DC0009CCAB7F7FF1F03C5477D9307F00F630465
:100DD000F5007D89F52EB72702409843C176FD16B0
:100DE000719B98C398431367170098C3B7170240C5
:100DF000D843D8C3D843758FD8C3D843B7060001AA
:100E0000D8C39843558F98C3984393166700E3DD82
:100E100006FED843B7160240719BD8C3D843136768
:100E20002700D8C32147DC42B18BE39EE7FE6FF079
:100E3000CFA7EFF2EFA6371702405C43370400203C
:100E40009146B18B130444016385D700A1466382A8
:100E5000D704B7376E01938707601CC0B7160240EE
:100E6000DC420840918313F7F700B707002093870F
:100E70004700BA978C23DC4293F5F50F93F70708E8
:100E80003357B50081E7EFF0EFA42A8718C06FF061
:100E9000CFA15C43B777DC02938707C07DBF01A079
:100EA0009701002093818197138181FE1305000A29
:100EB00097F5FF1F9385051517F6FF1F1306861478
:100EC00063FAC5008322050023A055001105910592
:100ED000E3EAC5FE170500001305856197F5FF1FBE
:100EE0009385451217F6FF1F1306461363FAC500D4
:100EF0008322050023A0550011059105E3EAC5FEF4
:100F000017F5FF1F13058511938541876377B5009A
:100F1000232005001105E36DB5FEB7220000938282
:100F20000288739002308D427390428097F2FFFFE7
:100F30009382420D93E2320073905230EFF05FE102
:100F40009702000093824284739012347300203021
:100F50005841032305004C453706014093070640DE
:100F60003E979346F3FFB1C583250640F58D2320B8
:100F7000B640D043F18ED4C31443B3E6660014C325
:100F8000184190479346F7FF758E90C7D047F18E72
:100F9000D4C7144541466399C6009447D98E94C777
:100FA000D447558FD8C78280B6979443558F98C33E
:100FB00082801C43F58F1CC38280B70701401387D2
:100FC000074083A70740584B698F09C77D8D33358C
:100FD000A000828001458280B707014023AAA74074
:100FE0008280B707674537270240938737125CC373
:100FF000B797EFCD9387B79A5CC3828037270240BB
:101000001C4B93E707081CCB8280B7270240C8C758
:101010008280372702405C470545858B91E748472A
:101020004189133515000D058280EFF26F872A8400
:10103000CD3785476318F50019E0154529A0D13F44
:101040007D14C5BF7DD86FF04F86EFF26F85AA84FF
:1010500037050B00D93F91476313F502372402404F
:101060001C4837050B0093E727001CC844C81C48E0
:1010700093E707041CC8553F1C48F59B1CC86FF03C
:10108000CF82EFF2EF817111AA8409652EC0713F02
:1010900091478245631EF500372402401C480965CC
:1010A00093E717001CC88EA049371C48F99B1CC841
:1010B00011016FE09FFF944593F7060193F2F6004C
:1010C00081C7DC41B3E2F20083D3050093F7F30F4D
:1010D000A5C303230500611122C226C08147130462
:1010E00080029304800405473316F70033F7C300EA
:1010F0006312E602939527003D473317B700134765
:10110000F7FF33736700B395B20033E36500639D67
:10111000860050C985072147E397E7FC1244232046
:101120006500824421018280E39696FE10C9DDB7F6
:10113000828008456D8D3335A000828019C20CC9AC
:1011400082804CC9828037070140144786058D474D
:10115000B397B70093C7F7FFF58F1CC71C47B315AC
:10116000B500DD8D0CC7828023A8A186828083A66E
:101170000187854718216390F6021C31639CD702D2
:101180003C219A0793E707F8B7E600E093F7F70FDB
:10119000BA962380F6408546935757003397E6006A
:1011A000544189CE938707048A07B7E600E0B697D3
:1011B00098C38280EDF33C219A07F9B7938707061D
:1011C000B7E600E08A07B69798C30F100000828048
:1011D000371702401C430E0593F777F05D8D08C367
:1011E000828099C5371702401C4F5D8D08CF8280E1
:1011F000B7170240984F1345F5FF798D88CF82804D
:1012000099C5371702405C4F5D8D48CF8280B71774
:101210000240D84F1345F5FF798DC8CF82801E213B
:1012200037370140130707C0C207C1836306E500D3
:10123000370700406316E500BA2193F7F7F8D98F16
:10124000FA2193F7F7CFC207C183D98F1EA1DE2100
:101250005EB59E211EB5B7370140938707C0631462
:10126000F5009C251EB985475EA982801E316577F1
:101270001307F7CFC207C183BD9BC207C1831EB14D
:101280001E31562103D38500C20713960601162D81
:10129000C18393F7F7FD758F96214182A206558F82
:1012A000B62142074183B3E666009206D58FB73672
:1012B0000140C207938606C0C183631ED502B625CE
:1012C00093F7F7F703D3C5009206D58FD621C2074F
:1012D000C183920693F7F7FBD58FFD769386F63F91
:1012E000F18EF225C207C183336666000A06D18EED
:1012F00013960601418252A11AADFA2118DD1EB1E2
:1013000082801A31FD77FD17F98F1EB10353050254
:101310005A215E2DE5769386F6CFFD8E9E2113161B
:101320000701BA21A207DD8EF977FD17B3F7670031
:1013300003D38500C2064182336767003207D98F25
:1013400037370140C207130707C0C182C183631B3F
:10135000E50071777D17718FD2251A06518F13160C
:1013600007014182FA2152A156AD38C11EB18280D7
:101370001E2189C593E717001EA18280C207C18381
:10138000F99BC207C183CDBF8357450491C521672F
:10139000D98F2312F5048280C607C583DDBF0EB541
:1013A00052A982804EB582800CDD82802CC1828061
:1013B000B3C7A5008D8B3307C50081E78D4763E771
:1013C000C702AA87637EE50A942185078505A38F56
:1013D000D7FEE3EBE7FE8280942185078505A38F86
:1013E000D7FEE3EBE7FE02441101828093763500DD
:1013F000AA8789CA942185078505A38FD7FE93F60E
:101400003700C5BF9376C7FF138606FE63F5C70690
:10141000711122C0C04903A3050083A38500C0CB7E
:10142000804D23A0670003A3450080CFC04D23A2B9
:10143000670083A2C50003A3050193854502C0CFC1
:1014400003A4C5FF23A4770023A6570023A86700A1
:101450009387470223AE87FEE3EEC7FAE3F3D7F89C
:1014600090419107910523AEC7FECDBF90419107F2
:10147000910523AEC7FEE3EBD7FEE3E7E7F48280F6
:101480008280000004000000010000000400000051
:101490000400000000000000100000000100000037
:1014A00002000000010000001000000081F80501AA
:1014B000017F609C0500000000000000C08000006B
:1014C000000000000000000002000000000000001A
:1014D000000000000000000000000000000000000C
:0C14E00000000000000000000000000000
:1014EC0001010100010203040506070801020304BF
:0814FC0005060708006CDC0284
:00000001FF
